:020000040000FA
:0608000083EF22F012005C
:06080800BBEF05F0120039
:0608180022EF04F01200C3
:06082A0002004845000039
:10083000DE0100000200000045450000D901000073
:0408400003000000B1
:0C084400D8CFE4FFE0CFE4FFE46EDACF91
:10085000E4FFE2CFDAFFE9CFE4FFEACFE4FFF3CF32
:10086000E4FFF4CFE4FFE6529EA201D19E92030E74
:10087000386E0E50EA6A510FE96E010EEA22EF500F
:10088000385C30E10E50E96EEA6AD890E936EA3613
:10089000690EE926010EEA22EECF38F0EFCF39F0EB
:1008A00039C038F0396A3850D76E0E50E96EEA6AAE
:1008B000D890E936EA36690EE926010EEA22EECF33
:1008C00038F0EFCF39F03850D66EF28AF294D58EE8
:1008D0000E50EA6A510FE96E010EEA22040EEF6E25
:1008E0000E50106E020E386E0F50EA6A510FE96E0C
:1008F000010EEA22EF50385C49E10F50E96EEA6AD6
:10090000D890E936EA36690EE926010EEA22EE5061
:10091000ED1009E10F50EA6A510FE96E010EEA226B
:10092000010EEF6E33D0080E0F5C0CE2070E0F14B1
:10093000386E010E385204E0E846FE0B3806FCE142
:1009400089121AD0100E0F5C0CE2070E0F14386ECD
:10095000010E385204E0E846FE0B3806FCE18A122C
:100960000BD0070E0F14386E010E385204E0E84623
:10097000FE0B3806FCE18B120F50EA6A510FE96E4C
:10098000010EEA22030EEF6E0F500E6E0F2A060EB6
:100990000F5C03E1080E0F6E0AD0130E0F5C03E12B
:1009A000160E0F6E04D0180E0F5C01E10F6A000ED8
:1009B000D8800254000E03542EE2112A000E122297
:1009C0000250115C0350125826E3116A126A030E9A
:1009D000065C1FE20450EA6A480FE96E010EEA2243
:1009E00080CFEFFF0450EA6A4B0FE96E010EEA2256
:1009F00081CFEFFF0450EA6A4E0FE96E010EEA2242
:100A000082CFEFFF042A030E045C01E3046A062A86
:100A100002D0026A036A000ED8800754000E085400
:100A200019E20C50000816E2132A000E1422075097
:100A3000135C085014580EE3136A146A030E0B5C1F
:100A400007E2092A030E095C01E3096A0B2A02D0B6
:100A5000076A086A0C5000080AE2156A1550040D6E
:100A6000F328C26E9E9C9F9C9D8CC280C2829EACCD
:100A70002DD09E9CC4503C6E3CC03DF03C6AC3509F
:100A800000013C103A6E3DC03BF01550060DF3CF0F
:100A900038F0F4CF39F0000E3826010E3922095013
:100AA000020D3850F324E96E3950F420EA6E3AC052
:100AB000EEFF3BC0EDFF152A0C50155C02E39D9C38
:100AC00005D01550040DF328C26EC282F2A442D0A4
:100AD000D59EF294F29A040E386E1050EA6A510FC5
:100AE000E96E010EEA22EF50385C34E1080E105C2A
:100AF0000DE2070E1014386E010E385204E0E8467D
:100B0000FE0B3806FCE1E81C89161CD0100E105CA8
:100B10000DE2070E1014386E010E385204E0E8465C
:100B2000FE0B3806FCE1E81C8A160CD0070E1014E8
:100B3000386E010E385204E0E846FE0B3806FCE140
:100B4000E81C8B161050EA6A510FE96E010EEA227A
:100B5000020EEF6EE552E5CFF4FFE5CFF3FFE5CFF0
:100B6000EAFFE5CFE9FFE5CFDAFFE550E5CFE0FFAB
:100B7000E5CFD8FF1000DACFE4FFE2CFDAFFE6528C
:100B8000E552E5CFDAFF1100D9CFE6FFE1CFD9FF7B
:100B9000020EE126896A92680F0EC16EC2900C6A3D
:100BA000070EB46E8A6A93688B6A9468FC0E8B1683
:100BB000FC0E941694840101010EC16F0101DE69DF
:100BC000DF690A6A096A0B6A056A046A066A026AC8
:100BD000036A076A086A116A126A136A146A156A54
:100BE000CA82CA80CA9CCA9ACA88CA96FA0ECB6EB2
:100BF000DF6ADFCF2AF00C0EE76E2A18E8AE02D0CB
:100C0000E73402D0E7502A5C38E2010EDB6A010EBD
:100C1000DBCF2AF0030EE76E2A18E8AE02D0E734E5
:100C200002D0E7502A5C27E2DFCF2AF02B6A2ABEE7
:100C30002B68060E2B02F3CF2BF0060E2A02F3CF01
:100C40002AF0F4502B26000E2A26010E2B22010E2C
:100C5000DBCF2CF02D6A2CBE2D68D8902C362D368B
:100C60002A502C24E96E2B502D20EA6EEE6AED6A94
:100C7000010EDB2ACCD7DF2ABCD70101BB6B0101F7
:100C8000BC6B0101B96B0101BA6B0101BD6B0101C4
:100C9000BE6B0101BF6B0101C06B0E6A0F6A106A67
:100CA000DF6ADFCF2AF0180EE76E2A18E8AE02D00E
:100CB000E73402D0E7502A5C1BE2DFCFE9FFEA6AA3
:100CC000E9BEEA68D890E936EA36690EE926010EEF
:100CD000EA22EE6AED6ADFCFE9FFEA6AE9BEEA6876
:100CE000510EE926010EEA22010EEF6EDF2AD9D756
:100CF000D586D59AD59CF294F29AF194D08ECA9466
:100D00009D829F92F28EF28CCA84020EE15C02E216
:100D1000E16AE552E16EE552E7CFD9FF1200D9CF83
:100D2000E6FFE1CFD9FF020EE126010EDB6A0101E9
:100D3000996B0DEC13F0060E0101D55D03E36D50C8
:100D4000020B01E005D10650000809E202EC0BF0AD
:100D5000052A030E055C01E1056A0606F4D70B506F
:100D6000000809E22EEC0BF00A2A030E0A5C01E1EE
:100D70000A6A0B06F4D7040118BF65D00101996B0C
:100D8000040119510101995D53E201019951EA6A87
:100D9000080FE96E050EEA22EFCFDFFF0101D951FE
:100DA0001CE10D0E2A6EDF502A5C05E00A0E2B6E48
:100DB000DF502B5C12E10101010ED96F0101BB5123
:100DC000EA6A400FE96E020EEA220D0EEF6E010193
:100DD000BB2BDE52010EDD6E15D00D0EDF5C11E077
:100DE0000A0EDF5C0EE00101BB51EA6A400FE96EBA
:100DF000020EEA22DFCFEFFF0101D96B0101BB2B0D
:100E000001D013D0400E0101BB5D02E10101BB6BBB
:100E10000101BC510101BB5D02E10D8609D0010E4B
:100E2000DB5003E015D9010EDB6A0101992BA8D72D
:100E30000401400E196F400E040118170401187DBB
:100E4000880E040118130D5001E181D00DA010D0BF
:100E5000AB0E2A6E3F0E2B6E2C6A2AC0E6FF2BC00B
:100E6000E6FF2CC0E6FF05EC21F0E552E552E55225
:100E70000DA210D0A50E2A6E3F0E2B6E2C6A2AC032
:100E8000E6FF2BC0E6FF2CC0E6FF05EC21F0E552A3
:100E9000E552E5520DA410D0890E2A6E3F0E2B6E3E
:100EA0002C6A2AC0E6FF2BC0E6FF2CC0E6FF05EC4B
:100EB00021F0E552E552E5520DA610D06D0E2A6ED6
:100EC0003F0E2B6E2C6A2AC0E6FF2BC0E6FF2CC01B
:100ED000E6FF05EC21F0E552E552E5520DA810D0F1
:100EE0004E0E2A6E3F0E2B6E2C6A2AC0E6FF2BC0D8
:100EF000E6FF2CC0E6FF05EC21F0E552E552E55295
:100F00000DAA00D00DAC10D02D0E2A6E3F0E2B6E08
:100F10002C6A2AC0E6FF2BC0E6FF2CC0E6FF05ECDA
:100F200021F0E552E552E5520DAE10D0140E2A6EB6
:100F30003F0E2B6E2C6A2AC0E6FF2BC0E6FF2CC0AA
:100F4000E6FF05EC21F0E552E552E5520D6A35D891
:100F5000020EE15C02E2E16AE552E16EE552E7CFA2
:100F6000D9FF1200D9CFE6FFE1CFD9FF0101B95176
:100F7000EA6A000FE96E020EEA22FE0EDBCFEFFFF7
:100F80000101B92B400E0101B95D02E10101B96B0C
:100F90000101BA510101B95D01E10D84FE0EDBCF03
:100FA0002AF02B6A2ABE2B682AC0F3FF2BC0F4FF5D
:100FB00000D0E552E7CFD9FF1200D9CFE6FFE1CF4D
:100FC000D9FFE65201019A513EE10101B9510101F7
:100FD000BA5D39E00101BA510101D880B9551AE270
:100FE0000101BA510101B95DDF6E0101BA51010180
:100FF0009B6F9C6B000E01019B27020E01019C233D
:10100000DFCF9FF10101A06B0101010E9A6FB9C101
:10101000BAF119D0400E0101D880BA55DF6E010136
:10102000BA5101019B6F9C6B000E01019B27020EC0
:1010300001019C23DFCF9FF10101A06B0101010E93
:101040009A6F0101BA6BE552E552E7CFD9FF120062
:10105000D9CFE6FFE1CFD9FF040EE126DE6ADD6AD3
:10106000020EDB6A030EDB6A0101BC51EA6A400F23
:10107000E96E020EEA22EF50E66EE66AFEEC21F01F
:10108000E552E552020EF3CFDBFF0101BC2B400E0F
:101090000101BC5D02E10101BC6B020EDB50DE6EA2
:1010A000DD6A0101BC51EA6A400FE96E020EEA22D4
:1010B000EF502C0835E00101BC51EA6A400FE96E9F
:1010C000020EEA22EF500D082BE00101BC51EA6A42
:1010D000400FE96E020EEA22EF50E66EE66AFEEC81
:1010E00021F0E552E552030EF3CFDBFF0101BC2BEB
:1010F000400E0101BC5D02E10101BC6B020EDBCFC1
:101100002CF02CC02DF02C6A030EDB5000012C2497
:101110002A6E000E2D202B6E2AC0DEFF2BC0DDFFB5
:10112000000EDBCF1EF0010EDBCF1FF0490E1E18A4
:1011300002E1430E1F1801E1D7D0490E1E1802E14B
:10114000520E1F1801E1CDD0490E1E1802E1530EB8
:101150001F1801E1C3D0530E1E1802E1430E1F18E1
:1011600001E1B9D0530E1E1802E1520E1F1801E121
:10117000AFD0530E1E1802E1530E1F1801E1A5D087
:10118000530E1E1802E1420E1F1801E19BD0430EC0
:101190001E1802E1420E1F1801E191D0430E1E18E5
:1011A00002E1520E1F1801E187D04F0E1E1802E116
:1011B000420E1F1801E17DD0570E1E1802E14D0EA0
:1011C0001F1875E0520E1E1802E14D0E1F186DE03B
:1011D000440E1E1802E1500E1F1865E04F0E1E1837
:1011E00002E1500E1F185DE0490E1E1802E1500E7C
:1011F0001F1855E0580E1E1802E1540E1F184CE03F
:10120000540E1E1801E11F5045E0410E1E1801E169
:101210001F503EE0560E1E1801E11F5037E0490EE8
:101220001E1801E11F5030E04F0E1E1801E11F5043
:1012300029E0550E1E1802E1430E1F1821E0580E3A
:101240001E1802E1430E1F1818E0430E1E1801E19C
:101250001F5011E0520E1E1801E11F500AE0580EF7
:101260001E1802E1520E1F1801E041D0BCEC0DF037
:101270007DD0B3D87BD036D979D0BEEC0DF076D006
:10128000B0D874D08CD972D0BDD970D0D6D96ED028
:10129000E5D96CD0E6D86AD0BAEC0DF067D051DB56
:1012A00065D0CFDB63D0B1DA61D06EDA5FD037DAE8
:1012B0005DD0B0EC0EF05AD0C0EC0DF057D069EC18
:1012C0000EF054D0F7EC0FF051D0B3EC10F04ED03C
:1012D000B6EC10F04BD0B9EC10F048D0BCEC10F0EC
:1012E00045D0BFEC10F042D0C2EC10F03FD0030E5E
:1012F000DB501AE1020EDBCFE6FFE66A020EDBCF1F
:10130000E6FFE66AF10E2A6E3E0E2B6E2C6A2AC0AC
:10131000E6FF2BC0E6FF2CC0E6FF05EC21F02D6EAA
:10132000070EE15E2D5021D0030EDBCFE6FFE66A0B
:10133000020EDBCFE6FFE66A030EDBCFE6FFE66ACE
:10134000020EDBCFE6FFE66AC90E2A6E3E0E2B6E5A
:101350002C6A2AC0E6FF2BC0E6FF2CC0E6FF05EC96
:1013600021F02D6E0B0EE15E2D5000D00101BC511D
:10137000EA6A400FE96E020EEA22EF500D080DE016
:101380000D500BE1520E2A6E2B6ADF502A1803E132
:10139000DE52DD502B1801E00D8EBBC1BCF1040EF6
:1013A000E15C02E2E16AE552E16EE552E7CFD9FF86
:1013B00012000101C15110E0C80E2A6E440E2B6EBE
:1013C0002C6A2AC0E6FF2BC0E6FF2CC0E6FF05EC26
:1013D00021F0E552E552E5521200C4EC05F0E9DFD8
:1013E0001200D9CFE6FFE1CFD9FF030EE126010EAF
:1013F000E66EC5EC10F0E5521D50DF6E020EE66E93
:10140000C5EC10F0E552DE521DC0DEFF1EC0DDFF50
:10141000DD520D5001E01BD0DF0418E1D950010F5F
:10142000E96EDACFEAFFEE50ED100BE0010E2A6E06
:101430002B6A010EDB502A1803E1020EDB502B1839
:1014400004E1010EDBCFC1F101D00D8CB2DF030E40
:10145000E15C02E2E16AE552E16EE552E7CFD9FFD5
:101460001200D9CFE6FFE1CFD9FF030EE126020E2D
:10147000DB6A030EE66EC5EC10F0E5521DC000F00D
:101480001EC001F0010EE66EC5EC10F0E552020E32
:101490001DC0DBFF0D5001E01BD0020EDB500CE144
:1014A0000050011003E1026A036A05D0CA8400C03B
:1014B00002F001C003F00BD00050011003E1076AF5
:1014C000086A05D0CA8400C007F001C008F071DFC7
:1014D000030EE15C02E2E16AE552E16EE552E7CF1C
:1014E000D9FF1200D9CFE6FFE1CFD9FF040EE126E4
:1014F000010EE66EC5EC10F0E5521D50DF6E010ED8
:10150000E66EC5EC10F0E552010E1DC0DBFF010ECA
:10151000E66EC5EC10F0E552020E1DC0DBFF010EB9
:10152000E66EC5EC10F0E552030E1DC0DBFF0D505A
:1015300001E02BD0DF50926E010EDB50936E020E55
:10154000DB50946E030EDB500C0805E20C0EF36EBC
:10155000030EF3CFDBFF030EDB5005E10F0EC16E70
:10156000C2900C6A11D00C6AC26A030EDBCFE6FF90
:101570000F0EE552D880E754C16EBE0EC06EC28019
:10158000030EDB500C6ECA8414DF040EE15C02E231
:10159000E16AE552E16EE552E7CFD9FF1200D9CFFB
:1015A000E6FFE1CFD9FF030EE126010EE66EC5ECA2
:1015B00010F0E5521D50DF6E010EE66EC5EC10F026
:1015C000E552010E1DC0DBFF010EE66EC5EC10F00A
:1015D000E552020E1DC0DBFF0D5001E009D0DF50C7
:1015E000896E010EDB508A6E020EDB508B6EE1DEDF
:1015F000030EE15C02E2E16AE552E16EE552E7CFFB
:10160000D9FF12008250E66EE66A8150E66EE66A05
:101610008050E66EE66AB60E2A6E3E0E2B6E2C6A7F
:101620002AC0E6FF2BC0E6FF2CC0E6FF05EC21F048
:101630002D6E090EE15E2D501200D00E2A6E440E62
:101640002B6E2C6A2AC0E6FF2BC0E6FF2CC0E6FFFB
:1016500005EC21F0E552E552E5521200D9CFE6FF44
:10166000E1CFD9FFE652DF6AB40E2A6E3E0E2B6E32
:101670002C6A2AC0E6FF2BC0E6FF2CC0E6FF05EC73
:1016800021F0E552E552E552DF6A0C50DF5C32E2B0
:10169000DFCF2AF02B6A2ABE2B68060E2B02F3CF6F
:1016A0002BF0060E2A02F3CF2AF0F4502B26000E60
:1016B0002A26010E2B220A50020D2A50F324E96E2D
:1016C0002B50F420EA6EEECFE6FFEFCFE6FFAE0E32
:1016D0002C6E3E0E2D6E2E6A2CC0E6FF2DC0E6FF4E
:1016E0002EC0E6FF05EC21F02F6E050EE15E2F50B7
:1016F000DF2ACBD7CD0E2A6E440E2B6E2C6A2AC061
:10170000E6FF2BC0E6FF2CC0E6FF05EC21F0E5521A
:10171000E552E552E552E552E7CFD9FF1200D9CFA5
:10172000E6FFE1CFD9FF030EE126030EE66EC5EC1E
:1017300010F0E5521DC0DEFF1EC0DDFF010EE66E9B
:10174000C5EC10F0E552020E1DC0DBFF0D5001E0AC
:1017500011D0DECF2AF0DDCF2BF0000E2A5C100E68
:101760002B5807E2DECFE9FFDDCFEAFF020EDBCF29
:10177000EFFF1FDE030EE15C02E2E16AE552E16E7B
:10178000E552E7CFD9FF1200D9CFE6FFE1CFD9FF6D
:10179000030EE126030EE66EC5EC10F0E5521DC007
:1017A000DEFF1EC0DDFF0D5001E025D0DECF2AF0A8
:1017B000DDCF2BF0000E2A5C100E2B5807E2DECF97
:1017C000E9FFDDCFEAFF020EEFCFDBFF020EDBCF3A
:1017D000E6FFE66AA40E2A6E3E0E2B6E2C6A2AC025
:1017E000E6FF2BC0E6FF2CC0E6FF05EC21F02D6ED6
:1017F000050EE15E2D50030EE15C02E2E16AE55266
:10180000E16EE552E7CFD9FF1200D9CFE6FFE1CF75
:10181000D9FF030EE126050EE66EC5EC10F0E55289
:101820001D50DF6E010EE66EC5EC10F0E552010EA4
:101830001DC0DBFF010EE66EC5EC10F0E552020E96
:101840001DC0DBFF0D5001E072D0020EDB5001081D
:1018500002E20D8C6CD0010EDB50070802E20D8C09
:1018600066D0410E2A6EDF502A5C1CE1020EDB506E
:101870000DE1010EF36E010EDB5004E0D890F3365B
:10188000E806FCE1F350E81C92160BD0010EF36E53
:10189000010EDB5004E0D890F336E806FCE1F3508B
:1018A000921244D0420E2A6EDF502A5C1CE1020ED6
:1018B000DB500DE1010EF36E010EDB5004E0D89019
:1018C000F336E806FCE1F350E81C93160BD0010E4A
:1018D000F36E010EDB5004E0D890F336E806FCE12D
:1018E000F350931223D0430E2A6EDF502A5C1CE182
:1018F000020EDB500DE1010EF36E010EDB5004E031
:10190000D890F336E806FCE1F350E81C94160BD0AF
:10191000010EF36E010EDB5004E0D890F336E806BA
:10192000FCE1F350941202D00D8C01D042DD030E85
:10193000E15C02E2E16AE552E16EE552E7CFD9FFF0
:101940001200D9CFE6FFE1CFD9FF030EE126020E48
:10195000DB6A050EE66EC5EC10F0E5521D50DF6E39
:10196000010EE66EC5EC10F0E552010E1DC0DBFF66
:101970000D5001E05CD0010EDB50070802E20D8C37
:1019800056D0410E2A6EDF502A5C10E1010EF36E34
:10199000010EDB5004E0D890F336E806FCE1F3508A
:1019A0008014E76E020EE7CFDBFF2CD0420E2A6ECA
:1019B000DF502A5C10E1010EF36E010EDB5004E0F3
:1019C000D890F336E806FCE1F3508114E76E020E7E
:1019D000E7CFDBFF17D0430E2A6EDF502A5C10E101
:1019E000010EF36E010EDB5004E0D890F336E806EA
:1019F000FCE1F3508214E76E020EE7CFDBFF02D06A
:101A00000D8C15D0020EDBCFE6FFE66A9B0E2A6E28
:101A10003E0E2B6E2C6A2AC0E6FF2BC0E6FF2CC0C0
:101A2000E6FF05EC21F02D6E050EE15E2D50030E54
:101A3000E15C02E2E16AE552E16EE552E7CFD9FFEF
:101A40001200D9CFE6FFE1CFD9FF030EE126050E44
:101A5000E66E9BDBE5521D50DF6E010EE66E95DBF8
:101A6000E552010E1DC0DBFF010EE66E8EDBE55276
:101A7000020E1DC0DBFF0D5001E072D0020EDB50E4
:101A8000010802E20D8C6CD0010EDB50070802E267
:101A90000D8C66D0410E2A6EDF502A5C1CE1020ECE
:101AA000DB500DE1010EF36E010EDB5004E0D89027
:101AB000F336E806FCE1F350E81C89160BD0010E62
:101AC000F36E010EDB5004E0D890F336E806FCE13B
:101AD000F350891244D0420E2A6EDF502A5C1CE17A
:101AE000020EDB500DE1010EF36E010EDB5004E03F
:101AF000D890F336E806FCE1F350E81C8A160BD0C8
:101B0000010EF36E010EDB5004E0D890F336E806C8
:101B1000FCE1F3508A1223D0430E2A6EDF502A5C78
:101B20001CE1020EDB500DE1010EF36E010EDB50E5
:101B300004E0D890F336E806FCE1F350E81C8B167D
:101B40000BD0010EF36E010EDB5004E0D890F3369B
:101B5000E806FCE1F3508B1202D00D8C01D029DC99
:101B6000030EE15C02E2E16AE552E16EE552E7CF85
:101B7000D9FF12001EDC12001CDC12001ADC12005D
:101B8000D9CFE6FFE1CFD9FF060EE126050EE66EBE
:101B9000FCDAE5521D50DF6E010EE66EF6DAE55214
:101BA000010E1DC0DBFF030EE66EEFDAE552020EFA
:101BB0001DC0DBFF030E1EC0DBFF0D5001E07FD018
:101BC000D950020FE96EDACFEAFF720ED880EE54D8
:101BD0002E0EED5402E20D8C72D0020EDBCF1EF001
:101BE000030EDBCF1FF0040E1EC0DBFF050E1FC06F
:101BF000DBFF2D682E682F6A2D0EE76E020EDBCFFD
:101C000030F0030EDBCF31F0E7503026000E3122EA
:101C1000326A30502D5C2A6E31502E582B6E325065
:101C20002F582C6E020E2AC0DBFF030E2BC0DBFFE9
:101C3000010EDB50070802E20D8C41D0410E2A6EE6
:101C4000DF502A5C02E1DF6A12D0420E2A6EDF50BA
:101C50002A5C03E1080EDF6E0AD0430E2A6EDF50C5
:101C60002A5C03E1100EDF6E02D00D8C28D0010E2D
:101C7000DB50DF24E96EEA6AD890E936EA36690E6D
:101C8000E926010EEA22020EDBCFEEFF030EDBCFC8
:101C9000EDFF010EDB50DF24EA6A510FE96E010E01
:101CA000EA22EF040AE1010EDB50DF24EA6A510F59
:101CB000E96E010EEA22020EEF6ED9EC09F0060E73
:101CC000E15C02E2E16AE552E16EE552E7CFD9FF5D
:101CD0001200D9CFE6FFE1CFD9FF050EE126010EB4
:101CE000E66E53DAE5521D50DF6E010EE66E4DDAF8
:101CF000E552020E1DC0DBFF010EE66E46DAE5522C
:101D0000030E1DC0DBFF010EE66E3FDAE552010E49
:101D10001DC0DBFF010EE66E38DAE552040E1DC071
:101D2000DBFF0D5001E012D0DFCFB4F1020EDBCFAC
:101D3000B6F1010EDBCFB5F1030EDBCFB7F1040E28
:101D4000DBCFB8F1B4C189FFD9EC09F0050EE15C35
:101D500002E2E16AE552E16EE552E7CFD9FF1200F7
:101D6000D9CFE6FFE1CFD9FF040EE126030EDB6AEF
:101D70000101BC51EA6A400FE96E020EEA22EF50FF
:101D80002C081DE00101BC51EA6A400FE96E020E09
:101D9000EA22EF50E66EE66A740E2A6E3E0E2B6E55
:101DA0002C6A2AC0E6FF2BC0E6FF2CC0E6FF05EC3C
:101DB00021F02D6E050EE15E2D500D8A0ED1010130
:101DC000BC2B400E0101BC5D02E10101BC6BB4C142
:101DD00089FF0101B51D89142A6E891C0101B51501
:101DE0002A10E76E010EE7CFDBFF0101BC51EA6A62
:101DF000400FE96E020EEA22EF500D0801E1EBD030
:101E00000101BC51EA6A400FE96E020EEA22EF506E
:101E1000E66EE66AFEEC21F0E552E552020EF3CFE3
:101E2000DBFF300EF36E020EDBCFF4FFF350F45CF9
:101E30000FE3020EDB5039080BE3300E2A6E020E60
:101E4000DBCFE7FF2A50E75E020EE7CFDBFF19D0BA
:101E5000410EF36E020EDBCFF4FFF350F45C0FE3A0
:101E6000020EDB5046080BE3370E2A6E020EDBCF64
:101E7000E7FF2A50E75E020EE7CFDBFF02D00D8CB2
:101E8000ACD0020EDB38F00BDF6E0101BC2B400E34
:101E90000101BC5D02E10101BC6B0D0E2A6E010166
:101EA000BC51EA6A400FE96E020EEA22EF502A5C4A
:101EB00002E10D8892D00101BC51EA6A400FE96E3F
:101EC000020EEA22EF50E66EE66AFEEC21F0E552E1
:101ED000E552020EF3CFDBFF300EF36E020EDBCFC6
:101EE000F4FFF350F45C0FE3020EDB5039080BE310
:101EF000300E2A6E020EDBCFE7FF2A50E75E020E9D
:101F0000E7CFDBFF19D0410EF36E020EDBCFF4FFFB
:101F1000F350F45C0FE3020EDB5046080BE3370E80
:101F20002A6E020EDBCFE7FF2A50E75E020EE7CFF4
:101F3000DBFF02D00D8C51D0020EDB50DF24DF6EB0
:101F40000101BC2B400E0101BC5D02E10101BC6B33
:101F5000DF508A6E010EDB50896E0101B85105E039
:101F6000B8C1E6FF8FEC22F0E552B4C189FF010150
:101F7000B75130E0030EB7C1DBFF0101B4510101DD
:101F8000B6152A6E0101B65180142A5C0BE1030ECE
:101F9000DB5008E000000000000000000000030E1D
:101FA000DB06EBD7030EB7C1DBFF0101B451010122
:101FB000B6152A6E0101B65180142A5C0BE0030E9F
:101FC000DB5008E000000000000000000000030EED
:101FD000DB06EBD70AD7D9EC09F0040EE15C02E28C
:101FE000E16AE552E16EE552E7CFD9FF1200D9CFA1
:101FF000E6FFE1CFD9FF050EE126030EDB6A040EF2
:10200000DB6A010EE66EC1D8E552040E1DC0DBFF8F
:10201000040EDB5004E0040EDB50380802E20D8CA5
:1020200098D00101BC51EA6A400FE96E020EEA2223
:10203000EF502C081DE00101BC51EA6A400FE96E27
:10204000020EEA22EF50E66EE66A740E2A6E3E0E2B
:102050002B6E2C6A2AC0E6FF2BC0E6FF2CC0E6FFE1
:1020600005EC21F02D6E050EE15E2D500D8A71D02C
:102070000101BC2B400E0101BC5D02E10101BC6B02
:10208000B4C189FF0101B51D89142A6E891C0101A3
:10209000B5152A10E76E010EE7CFDBFF040EDB500B
:1020A00056E00101BC51EA6A400FE96E020EEA22D5
:1020B000EFCFDFFF0101BC2B400E0101BC5D02E14F
:1020C0000101BC6B040EDB06DF508A6E010EDB5093
:1020D000896E0101B85105E0B8C1E6FF8FEC22F02E
:1020E000E552B4C189FF0101B75130E0030EB7C119
:1020F000DBFF0101B4510101B6152A6E0101B65191
:1021000080142A5C0BE1030EDB5008E000000000A5
:10211000000000000000030EDB06EBD7030EB7C182
:10212000DBFF0101B4510101B6152A6E0101B65160
:1021300080142A5C0BE0030EDB5008E00000000076
:10214000000000000000030EDB06EBD7A7D7D9EC98
:1021500009F0050EE15C02E2E16AE552E16EE5524A
:10216000E7CFD9FF1200D9EC09F01200D9EC09F041
:102170001200D9EC09F01200D9EC09F01200D9ECE8
:1021800009F01200D9EC09F01200D9CFE6FFE1CF37
:10219000D9FF040EE126030EDB6A0D0E2A6E010143
:1021A000BC51EA6A400FE96E020EEA22EF502A5C47
:1021B00005E10D881D6A1E6A1F6A93D10101BC5199
:1021C000EA6A400FE96E020EEA22EF502C0820E086
:1021D0000101BC51EA6A400FE96E020EEA22EF509B
:1021E000E66EE66A740E2A6E3E0E2B6E2C6A2AC0CC
:1021F000E6FF2BC0E6FF2CC0E6FF05EC21F02D6EBC
:10220000050EE15E2D500D8A1D6A1E6A1F6A69D196
:102210000101BC2B400E0101BC5D02E10101BC6B60
:102220002D0E2A6E0101BC51EA6A400FE96E020EC2
:10223000EA22EF502A5C28E1040E2B6EFE0EDB50E2
:102240002B5C22E0050E2C6EFE0EDB502C5C1CE09D
:10225000FE0EDB0406E0030E2A6EFE0EDB502A5C47
:1022600006E10D8C1D6A1E6A1F6A3BD10DD0010E5E
:10227000F36E030EF3CFDBFF0101BC2B400E010117
:10228000BC5D02E10101BC6B040E2A6EFE0EDB5048
:102290002A5C11E0050E2B6EFE0EDB502B5C0BE072
:1022A000050EE66ED9CFE6FFDACFE6FF24D9E55278
:1022B000E552E5523AD00101BC51EA6A400FE96E9D
:1022C000020EEA22EFCF2AF02B6A2C6A2AC0DFFF27
:1022D000010E2BC0DBFF020E2CC0DBFF050E2A6EA9
:1022E000FE0EDB502A5C19E1000EDBCFE6FF010E8B
:1022F000DBCFE6FFFEEC21F0E552E552F3CF2AF00A
:10230000F4CF2BF02C6A2BBE2C682AC0DFFF010E05
:102310002BC0DBFF020E2CC0DBFF0101BC2B400EEB
:102320000101BC5D02E10101BC6B030EDB5021E049
:10233000DFCF2AF0010EDBCF2BF0020EDBCF2CF02B
:102340002268236824682AC01DF02BC01EF02CC010
:102350001FF0D9EC1FF01AC02AF01BC02BF01CC0D4
:102360002CF02AC0DFFF010E2BC0DBFF020E2CC0B9
:10237000DBFFFE0EDB5026E1DFCF2AF0010EDBCFC4
:102380002BF0020EDBCF2CF02C34000E2C1807E6BD
:10239000D8807F0E2A54000E2B54000E2C5401E2DC
:1023A0008CD0D9CFE9FFDACFEAFF020ED880EB500C
:1023B000FF0A06E6800EEE5CFF0EEE58FF0EEF58A9
:1023C00001E27BD0FE0EDB0424E1DFCF2DF0010E15
:1023D000DBCF2EF0020EDBCF2FF02F34000E2F18A4
:1023E00007E6D880FF0E2D54000E2E54000E2F54F9
:1023F00064E3D9CFE9FFDACFEAFF020ED890EB50C1
:10240000000A06E6000EEE5C000EEE58000EEF58D5
:1024100054E3020E306EFE0EDB50305C24E1DFCF61
:1024200031F0010EDBCF32F0020EDBCF33F033346C
:10243000000E331807E6D880FF0E31547F0E325459
:10244000000E33543AE3D9CFE9FFDACFEAFF020EA8
:10245000D880EB50FF0A06E6000EEE5C800EEE58C8
:10246000FF0EEF582AE3030E346EFE0EDB50345C91
:1024700029E1DFCF35F0010EDBCF36F0020EDBCFE6
:1024800037F03734000E371807E6D880FF0E355482
:10249000FF0E3654000E375410E3D9CFE9FFDACFE0
:1024A000EAFF020ED890EB50000A06E6000EEE5C42
:1024B000000EEE58000EEF5805E20D8C1D6A1E6AE4
:1024C0001F6A0FD0DFCF2AF0010EDBCF2BF0020EF8
:1024D000DBCF2CF02AC01DF02BC01EF02CC01FF04B
:1024E00000D0040EE15C02E2E16AE552E16EE552E1
:1024F000E7CFD9FF1200D9CFE6FFE1CFD9FF020E17
:10250000E126FD0EDBCFE9FFFE0EDBCFEAFFEE6A30
:10251000EE6AEE6A010EDB6AFC0EDB50F36E010E12
:10252000DBCFF4FFF350F45C55E20101BC51EA6AE1
:10253000400FE96E020EEA22EFCFDFFF300EDF5CC4
:1025400044E3DF50390841E3FD0EDBCFE9FFFE0E27
:10255000DBCFEAFFEECF2DF0EECF2EF0EFCF2FF056
:102560000A0E226E236A246A2DC01DF02EC01EF0B2
:102570002FC01FF0D9EC1FF01AC02DF01BC02EF099
:102580001CC02FF0300EDF5C306E316A326A2D5085
:1025900030242A6E2E5031202B6E2F5032202C6E7C
:1025A000FD0EDBCFE9FFFE0EDBCFEAFF2AC0EEFF18
:1025B0002BC0EEFF2CC0EEFF0101BC2B400E010131
:1025C000BC5D02E10101BC6B02D0000E05D0010E22
:1025D000DB2AA2D7010E00D02A6E020EE15C02E2D5
:1025E000E16AE552E16E2A50E552E7CFD9FF1200C9
:1025F0000650E66EE66A680E2A6E3E0E2B6E2C6A58
:102600002AC0E6FF2BC0E6FF2CC0E6FF05EC21F058
:102610002D6E050EE15E2D5012000101DA51DB1125
:1026200005E10101500EDA6FC30EDB6F0101DA071D
:10263000000EDB5B0101D55108E0010E2A6E6D50E2
:10264000020B01E0010E2A5C02E18B901AD001011D
:10265000D5050CE0020E0101D55D08E0030E010175
:10266000D55D04E0050E0101D55D02E18B8009D046
:10267000060E0101D55D05E10101DA51DB1101E131
:102680008B70120082B403D0010E03D002D0000E72
:0426900000D0120064
:0C26940086EC18F0FB0EDBCFF3FFDB063A
:1026A000F35000090AE0D4EC18F0FA0E3FEC19F0F0
:1026B000F3E12B1CF1E1010E01D0000EB5EF18F093
:1026C00086EC18F03B0EE12402E3E168E652E16E8D
:1026D000010EDB6A020EDB6AF90EDBCFF6FFFA0EA3
:1026E000DBCFF7FFFB0EDBCFF8FF0800F550DF6E06
:1026F000DF5002E1D9EF17F0250EDF5C02E0CCEFEE
:1027000017F0030EDB6A040EDB6A050EDB6A060EA9
:10271000DB6A070EDB6AEEEC17F02D0EDF5C0CE0D7
:102720002B0EDF5C09E0200EDF5C06E0230EDF5C91
:1027300003E0300EDF5C1AE1DF50300A14E0130AC8
:102740000FE0030A0AE00B0A05E0060AE4E1030EC3
:10275000DB80E1D7030EDB82DED7030EDB84DBD721
:10276000030EDB86D8D7030EDB88D5D72A0EDF5CB5
:102770001BE1EAEC17F038EC18F010E0030EDB80F8
:102780001E681F68130EDBCF23F0140EDBCF24F07E
:1027900022EC20F0040E1CC0DBFF03D0130E21EC52
:1027A00018F0EEEC17F00BD0090EDB6A8FEC18F086
:1027B00003E003EC19F0FAD7090E21EC18F0030E30
:1027C000DBB0DB982E0EDF5C1BE1EEEC17F02A0E7F
:1027D000DF5C0BE1EAEC17F038EC18F003E1130EC4
:1027E00073EC18F0EEEC17F00BD0090EDB6A8FECEF
:1027F00018F003E003EC19F0FAD7090E73EC18F0A7
:10280000680EDF5C07E1EEEC17F0680EDF5C1DE19F
:10281000030E18D0740EDF5C17E07A0EDF5C14E054
:10282000480EDF5C06E0540EDF5C03E05A0EDF5C0E
:1028300002E1020E07D06C0EDF5C03E06A0EDF5C83
:1028400004E1010EC6EC18F0C9DBDF506E0A01E1AD
:102850007FD31E0A01E192D1200A01E18FD13F0A04
:1028600001E149D11A0A01E146D10D0A01E143D142
:10287000200A01E140D13A0A01E13DD1200A01E1FB
:102880003AD1260A01E135D10D0A01E132D11A0A05
:1028900001E1D9D0200A4AE0300A1FE0460A0EE0E2
:1028A000250A01E083D3D950F90FE96EFF0EDA2033
:1028B000EA6E010EEE5E000EEE5AEE5AD4EC18F0FF
:1028C000250EE66E95DB03E12B1C01E169D3D0EC0C
:1028D00018F001E26BD3DB2A69D3080EDB6A040E21
:1028E000DB50010806E2040EDB0498EC18F0DB5024
:1028F0008BDB080EDB5009E0030EDB50010B05E11A
:1029000072DB01E04DD3080EDB6A64DBEFCFDFFF43
:1029100048EC19F003E12B1C01E142D3D0EC18F094
:1029200001E3DB2A60DB01E141D33AD3070EDB5040
:1029300002080FE114EC19F0030EDBEC18F00E0E98
:10294000EECFDBFF0F0EEECFDBFF100EEECFDBFF87
:1029500020D0F70EDBCF2DF0F80EDBCF2EF0020EDD
:102960002D5E000E2E5AF70E2DC0DBFFF80E2EC086
:10297000DBFF2DC0E9FF2EC0EAFFCBEC18F02C6A7C
:102980000E0E2AC0DBFF0F0E2BC0DBFF100E2CC07B
:10299000DBFF0E0EDBCFE6FF0F0EDBCFE6FF100EE8
:1029A000DBCFE6FFD9EC21F0E552E552E552130EFC
:1029B0001DC0DBFF140E1EC0DBFF060EDB5005E062
:1029C000130E0FEC19F001E26ADB33EC19F002E2AE
:1029D000130E37DBF6EC18F006E0040E0FEC19F0DE
:1029E00002E2050E2EDB030EDBB005D0FCDA01E0BF
:1029F000D7D2080EDB6A090EDB6A0E0EDBCFF6FFBC
:102A00000F0EDBCFF7FF100EDBCFF8FF0800F550FD
:102A1000DF6EDF5014E039EC19F011E248EC19F0E8
:102A200003E12B1C01E1BCD2BBDB01E3DB2A090E75
:102A3000DB2AD9500E0FE96E000ECBDBE7D7D3DAD5
:102A400001E1B4D2ADD2C6DA110EEECFDBFF120E29
:102A5000EDCFDBFF110EDBCFE6FF120EDBCFE6FF83
:102A6000CBEC21F0E552E552130EF3CFDBFF140E51
:102A7000F4CFDBFF060EDB5004E0130ED0DB01E2E7
:102A80000EDB33EC19F002E2130EDBDAAFDB05E00C
:102A9000040EC5DB02E2050ED4DA030EDBB005D06E
:102AA000A2DA01E07DD2080EDB6A090EDB6A110EA4
:102AB000DBCFE9FF120EDBCFEAFFEFCFDFFFDF5006
:102AC00014E0D7DB12E2E4DB03E12B1C01E168D266
:102AD00067DB01E3DB2A090EDB2A110EDB2ADBCFE1
:102AE000E9FF120EE8E3DB2AE6D77DDA01E15ED2E8
:102AF00057D2030EDB8E070EDB0410E195DB040ECC
:102B00005ADB0A0EEECFDBFF0B0EEECFDBFF0C0E17
:102B1000EECFDBFF0D0EEECFDBFF6CD0070EDB50F0
:102B200003082CE1030EDBAE0DD0B2DA020E76DA2A
:102B3000EFCF2AF02B6A2C6A2D6A2AAE39D02B6887
:102B40002C6835D0F70EDBCF2BF0F80EDBCF2CF056
:102B5000020E2B5E000E2C5AF70E2BC0DBFFF80E78
:102B60002CC0DBFF2BC0E9FF2CC0EAFFEFCF2AF01F
:102B70000A0E2AC0DBFF0B0EDB6A38D0070EDB50D3
:102B8000020809E1030EDBAE04D059DB2CAE10D0F5
:102B90000ED055DB0DD0030EDBAE12D079DA020E6B
:102BA0003DDAF9DA2C6A2D6A2BAE02D02C682D683A
:102BB000E2DA0C0E2CC0DBFF0D0E2DC0DBFF1AD0AD
:102BC000F70EDBCF2CF0F80EDBCF2DF0020E2C5ED3
:102BD000000E2D5AF70E2CC0DBFFF80E2DC0DBFFC8
:102BE0002CC0E9FF2DC0EAFFD6DAC5DA0C0EDB6A8D
:102BF0000D0EDB6A060EDB5005E1010EF36E050ECD
:102C0000F3CFDBFF150EDB6A160EDB6AD950370FE8
:102C10002A6E000EDA202B6E390E2AC0DBFF3A0E28
:102C20002BC0DBFF380EDB6A080EDB6A0A0EAEDA59
:102C3000DF50780A12E0200A10E0280A0CE0200A8F
:102C40000AE03F0A06E00D0A02E0200A08E1020E4F
:102C500005D0080E03D0080EDF26100E97DA030EFB
:102C6000DBBE02D0DB92DB94DB50800B24E08ADAFF
:102C7000D890030EEB50000A08E6000EEE5C000E42
:102C8000EE58000EEE58000EEE5815E213DA2168E9
:102C900022682368246893EC21F00A0E18C0DBFF39
:102CA0000B0E19C0DBFF0C0E1AC0DBFF0D0E1BC094
:102CB000DBFF2D0E08D0030EDBA202D02B0E03D0BB
:102CC000DBA408D0200EF36E170EF3CFDBFF150E3A
:102CD000DB2A02D0170EDB6A050EDB5003E1B7D901
:102CE00001E189D0340E2A6E450E2B6E000E2C6E3B
:102CF000070EDBCF2DF02E6A2F6A306A2DC021F02F
:102D00002EC022F02FC023F030C024F0D3D924EC01
:102D100022F02A501824F36E2B501920F46E2C50F8
:102D20001A20F86EF4CFF7FFF3CFF6FF0800090E74
:102D3000F5CFDBFF580EDF5C0FE1610EF36E090E7D
:102D40007BD90AE3200E2A6E090EDBCFE7FF2A505B
:102D5000E75E090EE7CFDBFF070EDBCF2AF02B6A19
:102D60002C6A2D6A0FDA2AC021F02BC022F02CC069
:102D700023F02DC024F0EECF1CF0EECF1DF0EECFEF
:102D80001EF0EFCF1FF024EC22F01FC0EDFF1EC09D
:102D9000EDFF1DC0EDFF1CC0EFFF390EDBCFE9FFDB
:102DA000DB063A0EDBCFEAFF01E2DB06090EDBCFE2
:102DB000EFFF150EDB2A4BD995E1030EDBA61DD0E4
:102DC0006F0EDF5C06E1C1D918E3150EDB285BDA74
:102DD00014D0780EDF5C09E0580EDF5C06E0620E6E
:102DE000DF5C03E0420EDF5C08E1020EF36E160EBC
:102DF000F3CFDBFF02D0150EDB6A030EDB50100BA6
:102E00000EE0040EDBCF2AF0050EDB50D8802A54EA
:102E100006E2060EDB5003E1040EDB5034DA95D9EE
:102E20000AE2050EDBCFE7FF150EDB50E75E050E6D
:102E3000E7CFDBFF02D0050EDB6A040EDBCF2AF002
:102E4000160E45D9D8802A5414E2160EDBCFE6FFC1
:102E5000150EDBCFE6FF040EDBCFE6FF050EDB50E1
:102E6000E552E75CE552D880E754E552D880E75454
:102E70005FD9030EDB50010B0BE1080EDB5008E0BD
:102E8000B2D801E08DD0080EDB50BED8080EDB6A48
:102E9000170EDB5007E088D9170EF1D903E12B1C80
:102EA00001E17ED0160EDB5016E07ED9300EE66EC4
:102EB0009FD802E12B1C74E077D9DFCFE6FF51ECFD
:102EC00021F0E552E552E552F4CF2BF00001F31C5E
:102ED00002E12B1C65E0050EDBCF2AF0160EDB505D
:102EE000D8802A5409E2050EDBCFE7FF160EDB502F
:102EF000E75E050EE7CFDBFF300EE66E050ECBD9A1
:102F00004FE1390EDB2ADBCFE9FF3A0E01E3DB2A82
:102F1000DBCFEAFF090EEFCFDBFFDB500EE044D939
:102F2000090EADD902E12B1C3BE0390EDB2ADBCFC9
:102F3000E9FF3A0EEDE3DB2AEBD755D831E1160E67
:102F4000DBCFE6FF080EC3D8E552E7245DD82ED0CC
:102F5000070EDB50030A1CE0010A14E0030A07E035
:102F60007BD9DBCFEEFF020EDBCFEDFF1FD0F5D814
:102F70002F6A2DAE02D02E682F682CD8BCD82FC057
:102F8000EEFF14D0EAD82DBE2E6824D8B4D80ED0C7
:102F900063D9DBCFEFFF0AD07BD905E12B1C03E11E
:102FA000F368F46810D0FCD801E3DB2A79D975EF17
:102FB00013F0010EDBCF2AF0020EDBCF2BF02AC07C
:102FC000F3FF2BC0F4FF3B0EE15C02E2E16AE55245
:102FD000E16ECBD029D9020EDBEF18F061D90800E1
:102FE000F550DF6E1200200EE66E080E4BEF19F062
:102FF00051EC21F0E552E552E552F3CF2AF0F4CF3F
:103000002BF00001F31C12002A6E2B6AD950010F1D
:103010004DD92A50EE262B50ED2212002E5E000EC6
:103020002F5AF70E2EC0DBFFF80E2FC0DBFF2EC08D
:10303000E9FF2FC0EAFF1200DBCFF4FFF350F45C8E
:103040001200DB50E76E040EE7CFDBFF12000A0E22
:10305000DBCF2AF00B0EDBCF2BF00C0EDBCF2CF0EE
:103060000D0EDBCF2DF02A502B102C102D1012003E
:10307000130EEECFDBFF140EEDCFDBFF130EDBCF15
:103080002AF0140EDBCF2BF00001800E2B1412005F
:10309000F70EDBCF2EF0F80EDBCF2FF01200050E6F
:1030A000DB50E66ED950130F01D9E552E750EE6EB2
:1030B000ED6A12000A0EDBCF1CF00B0EDBCF1DF009
:1030C0000C0EDBCF1EF00D0EDBCF1FF01200DBCF9E
:1030D000E6FF150EDBCFE6FF050EDB50E552E724D9
:1030E000E552E7241200DB50CED8010EF36E060E37
:1030F000F3CFDBFF1200EE50EFCFEAFFE96E2CC0FA
:10310000EEFF2DC0EEFF2EC0EEFF1200D9CFE6FF7E
:10311000DACFE6FFE1CFD9FFE2CFDAFF1200DFCF4F
:10312000E6FFE66A12EC22F0E552E552F350120097
:10313000E76E080EE7CFDBFF1200EECF2AF0EECFEE
:103140002BF0EFCF2CF02D6A1200050EDBCF2AF00A
:10315000150EDB50D8802A541200010EDBCF2CF064
:10316000020EDBCF2DF02E6A1200E552E5CFDAFF1A
:10317000E7CFD9FF12000A0E2AC0DBFF0B0E2BC0CF
:10318000DBFF1200D9500A0F56EF19F0F36E070E4D
:10319000F3CFDBFF1200EECF2AF0EFCF2BF01200BF
:1031A000010EDB2A020E1200FC0EDBCFE6FFFD0E45
:1031B000DBCFE6FF12002A5E000E2B5AF70E2AC064
:1031C000DBFFF80E2BC0DBFF2AC0E9FF2BC0EAFFB4
:1031D0001200DA20EA6EEF2AEECFF6FF000EEF22A1
:1031E000EECFF7FFEF22EECFF8FF1200040EDBCF99
:1031F000E6FF130EDB50E552E75C9ADFDB5004DF9D
:10320000060EDB501200090EDB500A0DF350DF24CE
:10321000D00FE76E090EE7CFDBFFEEEF17F0DB50C4
:10322000F36E050E1CEF18F0F70EDBCF2AF0F80E48
:10323000DBCF2BF01200DFCFE6FFF8EF17F028DF2F
:10324000030EECDE9DEF18F04AEC13F0E552E55268
:10325000E552E55200091200BDDEEE50EFCFEAFF65
:10326000E96E010E1200130EDB50F36E040E1CEF1C
:1032700018F0040EDB50F36E090E1CEF18F0DBCFD4
:10328000E6FFF8EF17F0E76E050EE7CFDBFF120061
:103290008BDF1BEF19F0DBCFE6FF86DF24EF19F0A1
:1032A000D950F90FE96EFF0EE9EF18F0E96E000E44
:0632B000DA20EA6E1200B4
:0A32B600040120511F0B010801E084
:1032C00060D004012051600BE842E842E842E84245
:1032D000E842010801E055D00401245104E0040152
:1032E000240501E04ED004012151230A48E0010ADF
:1032F00040E0030A30E0010A25E0240A22E0070A40
:103300001FE0010A1CE0030A11E0010A01E038D0C5
:103310000101030ECE6F0101AC0ECF6F010ED06F15
:103320000101D6930101080ED36F2BD00101030ECA
:10333000CE6F0101AC0ED16F010ED26F22D021D021
:1033400020D01FD00101030ECE6F0101A10ED16F5D
:10335000010ED26F16D00101030ECE6F0101A10E36
:10336000CF6F010ED06F0101D6930101070ED36F0D
:1033700008D00101030ECE6F22C4A8F102D001D003
:1033800000D012000101A16BC20EA26F010EA36F4B
:10339000A46B0101A56B0101A66B0101080EA76FCB
:1033A00001019A6B0101996B1A0E726E1E0E736EFB
:1033B0000401000E166F050E176F0401400E146F06
:1033C0000401400E196F0401080E1A6F050E1B6FE1
:1033D0000401880E186F0401480E1E6F050E1F6F42
:1033E0000401400E1C6F1200D9CFE6FFE1CFD9FFD8
:1033F0000101996B040118BF39D0FC0EDBCF2AF014
:1034000004011951D8802A5403E2FC0E19C4DBFFD1
:103410000101996BFC0EDB500101995D1CE2010179
:103420009951EA6A080FE96E050EEA22EF50E66E3E
:1034300001019951E76EFD0EDBCFE9FFFE0EDBCFF8
:10344000EAFFE750E926000EEA22E552E750EF6E68
:103450000101992BDFD70401400E196F400E0401C2
:1034600018170401187D880E0401181301019951E1
:1034700000D0E552E7CFD9FF1200D9CFE6FFE1CF68
:10348000D9FFE65201019A5101E031D0DF6ADF2A0B
:10349000DF502A6E2B6A2A5002E1010E2B1801E13F
:1034A0000BD0FD0EDBCFE9FFDB2AFE0EDBCFEAFF00
:1034B00001E3DB2AEF50EBE1DF502A6E2B6AD95093
:1034C000FD0FE96EFF0EDA20EA6E2A50EE5E2B50F9
:1034D000ED5ADF06FD0EDBCF9BF1FE0EDBCF9CF13C
:1034E000DFCF9FF10101A06B0101010E9A6FE55240
:1034F000E552E7CFD9FF1200D9CFE6FFE1CFD9FFE0
:10350000E65201019A5101E033D0DF6ADF2ADF5031
:103510002A6E2B6AFF0E2A1801E12B5001E10CD014
:10352000FD0EDBCFF6FFDB2AFE0EDBCFF7FF01E35C
:10353000DB2A0800F550EAE1DF502A6E2B6AD950E9
:10354000FD0FE96EFF0EDA20EA6E2A50EE5E2B5078
:10355000ED5ADF06FD0EDBCF9BF1FE0EDBCF9CF1BB
:10356000DFCF9FF10101010EA06F0101010E9A6FE3
:10357000E552E552E7CFD9FF1200D9CFE6FFE1CF00
:10358000D9FFE65204011CBF7DD0030E01019A5DF4
:1035900002E101019A6B01019A5101E173D0020E1F
:1035A00001019A5D06E104011D6B0101030E9A6F92
:1035B00061D001019A055EE1400E2A6E2B6A01017D
:1035C0009F512A5C000E2B5803E2400EDF6E02D0A2
:1035D0009FC1DFFFDFCF1DF4DF5001019F5D0101BF
:1035E0009F6F0101480E9D6F050E9E6F0101A005A2
:1035F00018E1DF5015E09BC1F6FF9CC1F7FF080002
:10360000F5509DC1E9FF9EC1EAFFEF6E01019D2BC0
:10361000000E9E2301019B2B000E9C23DF06E9D7A1
:1036200016D0DF5014E09BC1E9FF9CC1EAFFEF50C8
:103630009DC1E9FF9EC1EAFFEF6E01019D2B000EC7
:103640009E2301019B2B000E9C23DF06EAD701017C
:103650009F5110E104011D512A6E2B6A400E2A1859
:1036600001E12B5004E10101020E9A6F03D0010128
:10367000030E9A6F400E04011C1704011C7D880E76
:0E36800004011C13E552E552E7CFD9FF1200FA
:02368E006C507E
:1036900002E0000E01D0010E00090BE00401005110
:1036A0003C0BE842E8420D0802E10CD801D042D8B8
:1036B00008D06C5002E0000E01D0010E040901E0B8
:1036C0004BD81200D9CFE6FFE1CFD9FFE652010176
:1036D000CD6B0101CE6B0101D36BD46BE4EC1CF01C
:1036E000DF6ADF502A6E2B6A010E2A5C000E2B580F
:1036F0001BE20101CE5101E017D0F76ADF34FE0B67
:10370000F736F66E690EF626410EF7220900F5CF60
:103710002AF00800F5CF2BF004D02BC0FAFF2A5076
:10372000F96EFBDFDF2ADDD7F0D8E552E552E7CFAF
:10373000D9FF1200020E0101CD5D0CE1A4D80401F5
:1037400000BD04D00401C80E006F03D00401880E30
:10375000006F01D029D91200040E0101D55D0CE1E2
:1037600022C46EFF6E50000804E20101050ED56F01
:1037700003D00101030ED56F0101CD050CE10DD879
:10378000040104BD04D00401C80E046F03D0040179
:10379000880E046F01D008D91200D9CFE6FFE1CF1F
:1037A000D9FF020EE1260101080ED35D000ED459A7
:1037B00005E2D3C1DEFFD4C1DDFF03D0080EDE6E0B
:1037C000DD6A0401049304010491010EDB5004013D
:1037D0000413DFCF05F4000EDB500101D35F010EAF
:1037E000DB500101D45B0101280ED16F040ED26FB2
:1037F0000101D6A320D0D9CFE9FFDACFEAFFEE50FE
:10380000ED1018E0CFC1F6FFD0C1F7FF0800F5506A
:10381000D1C1E9FFD2C1EAFFEF6E0101D12B000E49
:10382000D2230101CF2B000ED023DF06010E01E2CF
:10383000DB06E1D71ED0D9CFE9FFDACFEAFFEE50A1
:10384000ED1017E0CFC1E9FFD0C1EAFFEF50D1C1C1
:10385000E9FFD2C1EAFFEF6E0101D12B000ED223A6
:103860000101CF2B000ED023DF06010E01E2DB06A3
:10387000E2D7020EE15C02E2E16AE552E16EE55256
:10388000E7CFD9FF1200D9CFE6FFE1CFD9FF020E73
:10389000E126030E04010015E76E010EE7CFDBFF02
:1038A00001C4DFFFDE500101D327DD500101D42325
:1038B0000101280ECF6F040ED06FD9CFE9FFDACF08
:1038C000EAFFEE50ED1017E0CFC1E9FFD0C1EAFFEB
:1038D000EF50D1C1E9FFD2C1EAFFEF6E0101D12B58
:1038E000000ED2230101CF2B000ED023DF06010EE4
:1038F00001E2DB06E2D7020EE15C02E2E16AE55298
:10390000E16EE552E7CFD9FF12006D980101CE516B
:103910000FE10401080E016F0401200E026F040E76
:10392000036F0401840E006F0401840E046F3BD00A
:10393000040120AF25D00101D3510401265D01010E
:10394000D4510401275904E226C4D3F127C4D4F189
:1039500024DF0101010ECD6F0401080E016F040187
:10396000200E026F040E036F0401800E006F04012D
:10397000280E066F040E076F0401C80E046F13D0E3
:103980000101020ECD6F0401056B0401C80E046F26
:103990000401080E016F0401280E026F040E036F6C
:1039A0000401C80E006F12000101CD6B0401080E66
:1039B000016F0401200E026F040E036F0401880ED4
:0839C000006F0401046B12000A
:0839C80004012051600BE842EC
:1039D000E842E842E842E842000901E058D0040128
:1039E0002151070A53E00B0A51E0070A42E0010A9D
:1039F0002CE00B0A28E0020A26E0030A22E0080A6B
:103A000012E0010A0EE00F0A0AE0030A01E03ED0CC
:103A10000101010ECE6F0101040ED56F38D038D8E8
:103A200036D093D834D00101010ECE6F0101D70EEC
:103A3000CF6F010ED06F0101D6930101010ED36F3C
:103A400026D0ABD824D0F9D822D00101010ECE6FF8
:103A5000040124510101CF6FD06BD80E0101CF2793
:103A6000010E0101D0230101D6930101010ED36F94
:103A70000ED00101010ECE6F04012451EA6AD80F65
:103A8000E96E010EEA2222C4EFFF01D000D012003D
:103A9000800E0401205D58E104012351030A34E043
:103AA000010A10E0030A01E04DD00101010ECE6FC2
:103AB00001019E0ECF6F400ED06F120E0101D36F29
:103AC000D46B40D00101010ECE6F04012251F66E7D
:103AD000F76AD890F636F7365F0EF626410EF722D3
:103AE0000900F5CFCFF10A00F5CFD0F1020E0101A8
:103AF000F76ACF25F66ED051F7220900F5CFD3F142
:103B00000A00F5CFD4F11ED00101010ECE6F0401E1
:103B10002251F66EF76AD890F636F736630EF6261F
:103B2000410EF7220900F5CFCFF10A00F5CFD0F111
:103B3000CFC1F6FFD0C1F7FF0800F5500101D36FE8
:103B4000D46B00D00101D68312000101010ECE6FAB
:103B50000F0EE66E710EE66E0F0EE66E1FEC1FF096
:103B6000E552E552E552010EE66ED80EE66E010E04
:103B7000E66E1FEC1FF0E552E552E55222C4D7F184
:103B80000401225104E10101050ED56F05D00101A8
:103B9000060ED56FC2EC19F012000401286B040167
:103BA000296B040120511F0B020A14E0030A0EE0E6
:103BB000010A01E034D00101010ECE6F0401288119
:103BC0000101D6A102D00401288329D00101010EF0
:103BD000CE6F25D00101010ECE6F040124510F0BD1
:103BE000080DF3502B6A000F2A6E040E2B220401DD
:103BF0002451800B01E0010E040DF35001012A2431
:103C0000D16F000E2B20D26FD1C1E9FFD2C1EAFFE4
:103C1000EF50040B03E00401010E286F00D00101F6
:103C2000CE050AE10101280ECF6F040ED06F01010D
:103C3000D6930101020ED36F12000401220511E197
:103C4000040120511F0B00090CE10101010ECE6F90
:103C5000030E0401215D03E10101D68102D00101BF
:103C6000D691040122513EE1040120511F0B0208AC
:103C700039E1040124510F0B000934E00101010E68
:103C8000CE6F040124510F0B080DF3502B6A000F67
:103C90002A6E040E2B2204012451800B01E0010E38
:103CA000040DF35001012A24D16F000E2B20D26F96
:103CB000030E0401215D07E1840ED1C1E9FFD2C1E9
:103CC000EAFFEF6E0FD0040124AF06D0D1C1E9FFA7
:103CD000D2C1EAFFEF6A06D0880ED1C1E9FFD2C196
:063CE000EAFFEF6E120086
:0A3CE6006DA610D802D06DB614D8F8
:103CF0000101D50509E16DBA07D0686A696A698072
:103D000069880101020ED56F12006D6A696A6D86BD
:103D10000101010ED56F12006D6A696A0101D56B50
:103D20001200FADF12000101D55101E13AD06850CA
:103D3000040B04E06950040B01E03CD86DB231D0B3
:103D40006850010B04E06950010B01E056D868503F
:103D5000100B04E06950100B01E024D86850400BB0
:103D600004E06950400B01E03DD86850200B04E0AE
:103D70006950200B01E038D86850020B04E069500C
:103D8000020B01E038D8030E0101D55D01E209D034
:103D90006850080B06E06950080B03E047EC1BF085
:103DA00068961200698468986D82A19AA08A0300BF
:103DB000A09A12006D926994689412000101D6A134
:103DC00010D0F8DF6D840101080EDC6F070EDD6F87
:103DD0000101DC07000EDD5B0101DC51DD11F8E1C2
:103DE0006D941200689C120070A003D0D4EC1CF0FB
:103DF0007090689A1200689212006A6A686A9F0E50
:103E00006B6E7B0E696E6E6A0F0EE66E710EE66E5D
:103E10000F0EE66E14D8E552E552E552160E706E9E
:103E200068A602D06896FCD76D98D4EC1CF001010E
:103E3000D6910101D76B0101030ED56F1200D9CFC6
:103E4000E6FFE1CFD9FFFD0EDBCFE9FFFE0EDBCFB2
:103E5000EAFFFC0EDB5004E0EE6AFC0EDB06F9D74D
:083E6000E552E7CFD9FF120083
:083E68005374617475733D256C
:103E7000690D0A002135204572723A204E6565644D
:103E800020636F6D6D61206E6578742C20666F7590
:103E90006E643A20272563270D0A0050492C2531EE
:103EA000750D0A004D522C253033750D0A002C2556
:103EB000303475004100492C253033692C253033CE
:103EC000692C253033690D0A002138204572723A79
:103ED00020556E6B6E6F776E20636F6D6D616E64D3
:103EE0002027256325633A253258253258270D0AA5
:103EF000002138204572723A20556E6B6E6F776ED6
:103F000020636F6D6D616E64202725633A253258FA
:103F1000270D0A002137204572723A2045787472C5
:103F200061207061726D617465720D0A0021362026
:103F30004572723A20496E76616C696420706172D4
:103F4000616D7465722076616C75650D0A002134AF
:103F5000204572723A204D697373696E67207061F3
:103F600072616D657465722873290D0A0021332012
:103F70004572723A20525820427566666572206F0B
:103F800076657272756E0D0A002132204572723AA2
:103F900020545820427566666572206F766572728D
:103FA000756E0D0A002131200D0A002130200D0A06
:013FB0000010
:0E3FB2001FC029F01EC028F01DC027F01D50B2
:103FC0002202F4CF1BF0F3CF1AF01E502302F4CFDD
:103FD0001DF0F3CF1CF02202F3501B26F4501C22DC
:103FE000E86A1D2227502302F3501B26F4501C229E
:103FF000E86A1D221F502202F3501C26F4501D2295
:104000001F5023021E6AE86A1E22F3501D26F45038
:104010001E2227502402F3501C26F4501D221F6A32
:10402000E86A1E221F2228502402F3501D26F45055
:104030001E22E86A1F2229502402F3501E26F45043
:104040001F22000C1FC029F01EC028F01E502302A2
:10405000F4CF1DF0F3CF1CF01F502402F4CF1FF05B
:10406000F3CF1EF02302F3501D26F4501E22E86AFF
:104070001F2228502402F3501D26F4501E22E86A05
:104080001F2224AE48EF20F028501E5E29501F5AF0
:0E40900029AE000C23501E5E24501F5A000C57
:02409E0012010D
:1040A000000202000008D8040A000000010200011A
:1040B00009024300020100803209040000010202EB
:1040C0000100052400100104240202052406000159
:1040D000052401000107058203080002090401000C
:1040E000020A0000000705030240000007058302E2
:1040F0004000000403090434034D006900630072AA
:10410000006F0063006800690070002000540065C3
:1041100000630068006E006F006C006F006700793C
:1041200000200049006E0063002E00340343004469
:104130000043002000520053002D003200330032B3
:1041400000200045006D0075006C0061007400697E
:10415000006F006E002000440065006D006F00B02D
:0B41600040B040F340F7402B41B63266
:04416C002A0EF66EB3
:10417000080EF76E000EF86E01010900F550C86FC9
:104180000900F550C96F03E1C86701D03DD00900AF
:10419000F550C36F0900F550C46F0900F550C56FA5
:1041A00009000900F550E96E0900F550EA6E0900B2
:1041B00009000900F550C66F0900F550C76F0900E6
:1041C0000900F6CFCAF1F7CFCBF1F8CFCCF1C3C1DC
:1041D000F6FFC4C1F7FFC5C1F8FF0101C65302E1F4
:1041E000C75307E00900F550EE6EC607F8E2C707AF
:1041F000F9D7CAC1F6FFCBC1F7FFCCC1F8FF010167
:0A420000C807000EC95BBFD712000B
:06420A00D9CFE6FFDACF78
:10421000E6FFE1CFD9FFE2CFDAFFE652E652E652FF
:10422000E652D950FB0F2A6EFF0EDA202B6E2AC001
:10423000DEFFDD6EDECFE6FFDDCFE6FFFB0EDBCF80
:10424000E6FFFC0EDBCFE6FFFD0EDBCFE6FFDEC1B7
:10425000E6FFDFC1E6FF60EC13F02A6E070EE15CBB
:1042600002E2E16AE552E16E2A50020EF3CFDBFF73
:10427000030EF4CFDBFF020EDBCF2AF0030EDBCF01
:104280002BF02AC0F3FF2BC0F4FF040EE15C02E226
:10429000E16AE552E16EE552E5CFDAFFE7CFD9FFFB
:0242A00012000A
:0E42A200D9CFE6FFDACFE6FFE1CFD9FFE2CFBA
:1042B000DAFFFB0EDBCF2AF0FC0EDBCF2BF0000188
:1042C000800E2B141AE1FB0EDBCFE9FFFC0EDBCFD7
:1042D000EAFFEECFF3FFEDCFF4FFEE2A000EEF2260
:1042E000F3CFE9FFF4CFEAFFFD0EDBCFEFFFEF5096
:1042F0002B6AF36E2BC0F4FF10D0FB0EDB50FE08D0
:1043000006E1FD0EDBCFE6FF75EC22F005D0FD0ED9
:10431000DBCFE6FFB2EC07F0E552E552E5CFDAFF7E
:06432000E7CFD9FF1200F7
:0A4326001C502102F3CF18F0F4CF71
:1043300019F02202F3501926000EF4201A6E1C50B8
:104340002302F3501A26000EF4201B6E1C50240288
:10435000F3501B261D502102F3501926F4501A2247
:10436000000E1B221D502202F3501A26F4501B226D
:104370001D502302F3501B261E502102F3501A2613
:10438000F4501B221E502202F3501B261F50210204
:06439000F3501B26120091
:0A439600FE0EE3CFE9FFFF0EE3CFB8
:1043A000EAFFF36AF46AEE5203E0F34AF42AFBD719
:1043B0001200FF0EE3CFF8FFE552FF0EE3CFF7FF49
:1043C000E552FF0EE3CFF6FFE552E66AE66AE66ADB
:1043D0000900F55209E0FD0EE32A05E1FE0EE32A8D
:1043E00002E1FF0EE32AF4D7FD0EE3CF1DF0FE0E2F
:0C43F000E3CF1EF0FF0EE3CF1FF0120021
:0443FC00FF0EE124AB
:10440000E96EFF0EE220EA6EEDCFF4FFEFCFF3FF8F
:10441000F46607D0600EF36404D07B0EF36001D025
:10442000F39A1200F36AF46AFF0EE124E96EFF0EBC
:10443000E220EA6EED6607D02F0EEF6404D03A0E4C
:08444000EF6001D0F32A120025
:084448001B6A1A6A196A186A5E
:10445000200EE76ED8901C361D361E361F361836D5
:1044600019361A361B362150185C22501958235021
:104470001A5824501B5809E32150185E2250195A2B
:1044800023501A5A24501B5A1C2AE72EE4D7120034
:1044900005D811D88FEC06F0FCD712000F0EC11210
:1044A000140E6F6E0101D56B0101D66B0101D76B44
:1044B000C4EC05F0120073EC1EF06FBE02D093EC5A
:0844C0001EF0BDEC1AF0120021
:0844C8004F4B0D0A000D0A0024
:1044D00055425720465720442056657273696F6EC7
:0944E00020312E342E300D0A00AB
:0644EA00FF0EE350ACBA26
:1044F00004D0AF6AAB8EAC8A949CACA2FED7AD6EF2
:06450000F36EF46A1200E4
:0A45060013EE00F023EE00F0F86A57
:0E451000179CB6EC20F048EC22F0FDD712000C
:02451E00FF0E8E
:10452000E350E84E1200000000D000D000D0E82E8A
:04453000FAD71200A4
:0C453400303132333435363738396162AB
:054540006364656600E4
:0345450000000073
:02454800FEFF74
:00000001FF
